:1000000007C1A3C221C120C11FC11EC11DC11CC186
:100010001BC11AC119C118C117C116C115C114C11C
:1000200013C112C111C1040309045A03680061001D
:10003000660074006D0061006E006E0023007300A6
:100040006F00660074007700610072006500200098
:1000500028007700770077002E00740075002D00CF
:100060006300680065006D006E00690074007A002E
:100070002E00640065002F007E00680065006800A7
:10008000610029004403680023007300200046003B
:100090006C00790053007400690063006B002D0050
:1000A00045006D0070006600E4006E0067006500AA
:1000B0007200200066006500320020002800560013
:1000C00052004300500029003A03680065006800B0
:1000D00061004000680072007A002E007400750014
:1000E0002D006300680065006D006E0069007400FB
:1000F0007A002E00640065003A00300030003100C4
:1001000033001201100100000008C016DC270001B6
:100110000102030109022200010100800A09040012
:10012000000103000000092101010001223800073D
:100130000581030800101502495E6473382FD0C78B
:100140008C9BA1B6FDEA0111001122312A73001126
:10015000000126B30233C45144756677767746555D
:10016000045D6676667720110491222322330851BC
:1001700000132233233344554454267F6477545567
:1001800044556657E673C8918A99AABBAABA88B93A
:10019000089DBABBAABBCCCDCCDDCEFFEA7FCCDDBF
:1001A000CDDDE6BFEEFD889998992ABFAA9B889875
:1001B0008899A8BBEAB3CCDFC49DEFFFEEFFC85D12
:1001C000ECDDEEFFEEEFD780ACC281CAC19420987F
:1001D0002AC600E000C8F7C405010904A101150002
:1001E000250175019502050919012902810295066B
:1001F0008101050609211501250C37D91642004752
:100200002755420055026601F075089501B102C0FC
:1002100011241FBECFE5D4E0DEBFCDBF14BA10E07D
:10022000A0E6B0E0E0E5FCE002C005900D92A43647
:10023000B107D9F710E0A4E6B0E001C01D92A03AE2
:10024000B107E1F71AD403C5DBCE85B7826085BF5D
:100250008BB780648BBF8BE4809373008AE58093B7
:10026000720008951F93CF93DF93609183006350D2
:1002700067FDC8C080918000C3E9D0E0C81BD109E8
:1002800080917F008D3209F0ABC0683009F0B8C0B2
:1002900083EC809367008AE580936000109264008D
:1002A0008881807619F0CE01C4D386C09A811092DD
:1002B00070008981882321F41092710082E076C059
:1002C000853019F49093840070C0863009F059C0CD
:1002D0008B81813041F482E091E0909382008093A1
:1002E000810092E149C0823041F484E191E0909331
:1002F00082008093810092E23FC0833041F59923D0
:1003000041F486E290E0909382008093810094E033
:1003100033C0913041F48AE290E090938200809360
:1003200081009AE529C0923041F484E890E09093EE
:1003300082008093810094E41FC09330E1F488EC44
:1003400090E090938200809381009AE315C08132FF
:1003500041F484E591E0909382008093810099E0DC
:100360000BC0823241F488ED91E09093820080933B
:10037000810098E301C090E080E480936400892FBD
:100380001BC0883021F481E026E830E011C08930BC
:1003900019F49093860009C08A3011F481E006C0F8
:1003A0008B3019F48BE48093730080E020E730E019
:1003B0003093820020938100982F8F3F39F48881F9
:1003C00087FD9E8180E88093640007C08F81882329
:1003D00021F48E81891708F4982F9093610010C042
:1003E0008091640087FF0CC0CE0116D38F3F21F4AB
:1003F0008EE18093600004C0882311F010926100A8
:10040000109283008091600084FF46C0609161007B
:100410006F3F09F441C090916700693008F047C010
:100420001092610088E8982790936700662309F48A
:1004300047C020918100309182008091640086FF46
:100440000AC0962FF901A8E6B0E084918D93319609
:100450009150D9F708C0962FF901A8E6B0E0819134
:100460008D939150E1F76150C901860F911D6F5F27
:10047000019690938200809381007727162F88E65B
:1004800090E05FD01C5F1C3010F01CE003C08FEFC9
:10049000809361001093600094E180B38C70B1F49C
:1004A0009150D9F71092840010927E000FC06850CE
:1004B0006093610088E898279093670068E0B9CF5F
:1004C00060E088E690E03DD014E0E1CFDF91CF918D
:1004D0001F9108951F93DC01162F8091720084FFF5
:1004E00007C08091730098E889278093730003C048
:1004F0008AE580937200912FE4E7F0E08D9181937B
:1005000091501916DCF3612F84E790E01AD01C5F3C
:10051000109372001F910895A82FB92F80E090E0EA
:1005200041E050EA60956F5F58F42D9138EF8227D3
:100530009795879510F0842795273F5FC8F3F3CFF1
:100540000895EADF8D939D930895CF93CFB7CF930E
:10055000829BFECF829B09C0829B07C0829B05C005
:10056000829B03C0829B01C0A3C0DF93C091800027
:10057000DD27C957DF4F829B02C0DF91EBCF2F935E
:100580000F931F9300B32FEF02FB20F94F933F937C
:1005900010B34FEF012702FB21F93BE031C04E7F42
:1005A000012F10B3216028C0102F4D7F2260000062
:1005B00000B329C04B7F2460012F000010B32BC073
:1005C00010B3477F28602AC04F7E00B320612CC043
:1005D0004F7D10B320622FC04F7B00B3206432C028
:1005E000422700B349934FEF0000102712FB20F978
:1005F00010B31C70C9F1297F91F2012702FB21F988
:1006000000B3237F89F2315058F1102712FB22F9F1
:1006100010B3277E79F2012702FB23F92F7C81F2A8
:1006200000B3102712FB24F92F7971F200C010B328
:10063000012702FB25F92F7359F200C000B31027E0
:1006400012FB26F9223040F200C010B3012702FB52
:1006500027F9243028F64F77206810B30000F9CF2F
:1006600010E41ABF002719C03B503195C31BD0407E
:1006700010E41ABF0881033CF9F00B34E9F0209133
:100680007E001981110F1213EDCF4A81441F0936E4
:1006900041F10D3211F0013E29F7009385003F91A1
:1006A0004F911F910F912F91DF91CAB7C6FD50CF87
:1006B000CF91CFBFCF91189520918500222379F358
:1006C000109183001123A1F53430A2F130938300FF
:1006D00020937F00109180003BE0311B309380001D
:1006E00029C00091830001301CF50AE54F7049F4E0
:1006F0003091600034FD20C000936000C7E6D0E078
:100700001FC03091720034FD17C000937200C3E720
:10071000D0E016C0052710E002BB1FC0052722C08D
:10072000052727C005272CC0052710E002BB33C0D2
:100730004AE503C042ED01C0432FC4E1D0E032E0FE
:1007400011B31C60929A02B311BB5F935CE020E886
:1007500020FF052702BB279517951C3FD8F620FFE1
:100760000527279502BB17951C3FC0F620FF0527DC
:100770002795179502BB1C3F98F620FF0527279564
:1007800017951C3F02BB70F600C0499120FF05275A
:1007900002BB279517951C3F38F620FF05272795A4
:1007A00002BB17951C3F40F520FF0527279517959D
:1007B00002BB1C3F18F520FF0527279517951C3F06
:1007C00002BBF0F4242F3A9519F6037F5F9102BB28
:1007D000000010918400110FC651D04011F0109309
:1007E0007E0010E41ABF046011B3137F402F437FD3
:1007F00002BB11BB42BB53CF0527D2CF0527D7CFB2
:100800000527DCCFC2989FB9779BFECF9FB18FB9E8
:10081000779BFECF8FB1C29A0000C2980895809155
:1008200062002AE3829FC001112485569B45EADFBE
:100830000895CF93DF93C0E0D0E0E0E0F0E0EE0F6A
:10084000FF1FEA53FE4F85919491DCDF2196FE0154
:10085000C930D105A1F7E3DFDF91CF91089581E899
:100860009AECD0DF83E89AECCDDF0895E82FE69587
:10087000FF27EA5BFE4F949180FD02C0892F03C0E1
:10088000892F82958F7099278F7090700895EADC78
:10089000A895B49BFECF0895FADF80E090EBB2DF1D
:1008A000992708951F93F8DFE1DF182F1295107F25
:1008B000F3DFDCDF182B80916500812728E09CE8BE
:1008C00080FB86950EF489272A95D1F780936500E1
:1008D000812F99271F910895CF92DF92FF920F9356
:1008E0001F93CF93DF936C0110926500DBDF082F1D
:1008F000182F1F70E6010993F0906500D3DF082FD1
:100900001F5FC601810F911D11500196C817D907AD
:1009100091F7A5DFF0268F2D9927DF91CF911F91B9
:100920000F91FF90DF90CF900895B49903C020E01D
:1009300030E009C080EA90E0CFDF20E030E088239B
:1009400011F421E030E0C90108950F931F93082F9F
:100950009EDF1127C801986B55DF1F910F910895F5
:100960001F93CF93DF93182F80916500812728E094
:100970009CE880FB86950EF489272A95D1F7809311
:100980006500812F82958F70C6E3D1E0FE01E80FEC
:10099000F11DE4918E2FD9DF1F70C10FD11DFE0113
:1009A0008491D3DFDF91CF911F910895EF92FF9251
:1009B0001F93CF93DF937C018AEA98EB23DF8AEAC7
:1009C00098EB20DF88E792E81DDF8AEABEDF8DE240
:1009D000BCDF84EDBADF10926500F70110811F7053
:1009E000E7018991BDDF1F5FC701810F911D115084
:1009F0000196C817D907A9F780916500B1DF8AEA87
:100A0000A4DF45DF89ED92E8FDDE29DFDF91CF919C
:100A10001F91FF90EF900895FC01613039F48081BF
:100A200080936200A0EFBFEF082E05D181E090E037
:100A30000895FC01808180768032E1F481818130EB
:100A400089F48381813019F486E690E004C0833014
:100A500089F482E690E0909382008093810081E0A7
:100A600090E00895893031F48381833019F48FEF59
:100A700090E0089580E090E0089514B714BE80E8F7
:100A800088B9A99903C08EEF809363008FE188BB7A
:100A90008091630091E0892785BB83EF82BB8CE264
:100AA00087BB81E58DB99EB983E088BB81E092E880
:100AB000A9DE88E081BD13FF07C080B38C7021F0F0
:100AC000A89580EA85BF889580E885BFA0EFBFEF35
:100AD000AAD0802D282F3327822F81508C3010F4FC
:100AE0002093620083E084BB899AA3DE85E083BF04
:100AF00089ED92E887DEB3DE80E090E083DE8091CE
:100B0000630085BBA2DB78948895A89585B301E046
:100B1000802785BBA7DB80E58A95F1F785B3802721
:100B200085BBB49B48C01091630093E0F92E1F254C
:100B30008AE0E82EE0929E0080EA90E0CDDE8823F5
:100B4000C9F510278091A1008033A1F58091A00004
:100B5000813211F5909166008091A20089278370FF
:100B600080939D0098279093660080E18093A00079
:100B7000F092A10080EA90E019DF8091660088235E
:100B800011F084E601C080E080939F0083E0182785
:100B900085E080939E000EC0813861F49091A200A0
:100BA000892F81508C3030F49093620038DE1F25FD
:100BB000E0929E0015BB08B600FE25C081E088BF0C
:100BC00080919E00882341F0815080939E0088236D
:100BD00019F48091630085BB80919F00882399F070
:100BE000815080939F00882371F4809166008093E8
:100BF0009D00109266008091630093E0892785BB79
:100C000084E180939E008091720084FF7DCF80916B
:100C10009D00882309F478CF61E086E690E05ADCF5
:100C200010929D0071CFE199FECFBFBBAEBBE09AA1
:100C300011960DB20895E199FECFBFBBAEBB0DBAC0
:100C400011960FB6F894E29AE19A0FBE0895FFCF7D
:040C50005AFF03FD47
:00000001FF
